:1000000000308A0004280000FF238316900000308F
:100010008A001E2826308400000803191D2801309C
:10002000A100A001A00B1228A10B11284A30A000AA
:10003000A00B18281B28800B0F28080003081F3965
:1000400083001F1383161F109F101F119F1107306D
:100050008312990000308316850085018312850183
:100060000230A500FA30A6000A20A50B322805149C
:100070008316051002308312A500FA30A6000A206C
:10008000A50B3D2805108316051083123028630048
:02400E0084111B
:00000001FF
;PIC12F675
;CRC=AAB1  CREATED="18-oct.-22 16:59"
